S011000048656E64694374726C2E7372656396
S11300000C9434000C9451000C9451000C94510045
S11300100C9451000C9451000C9451000C94510018
S11300200C9451000C9451000C9451000C94510008
S11300300C9451000C94D8060C9451000C9451006B
S11300400C9451000C9451000C9491070C94870764
S11300500C947D070C9482000C9451000C94510074
S11300600C9451000C94510011241FBECFEFD8E022
S1130070DEBFCDBF12E0A0E0B1E0E0E7FCE102C0EA
S113008005900D92A235B107D9F722E0A2E5B2E0BE
S113009001C01D92A73DB207E1F70E94D1020C9462
S11300A0360E0C940000909363028093620228E160
S11300B031E041E050E060E170E084E592E00E94CC
S11300C01E01E4E6F0E080818E7F8083EAE7F0E0C1
S11300D08081876880830895ECE7F0E09081907FC9
S11300E090648F70982B9083EAE7F0E09081986495
S11300F090838093640281E090E090935302809314
S1130100520208951F920F920FB60F9211242F934B
S11301103F934F935F936F937F938F939F93AF938B
S1130120BF93EF93FF93CF93DF93CDB7DEB72597BC
S1130130DEBFCDBF1092530210925202809178001C
S11301402091790090917A00906190937A0092E0E6
S11301509983909164029A8390E0922B9C838B8381
S1130160BE016F5F7F4F80916202909163020E9493
S1130170630184E592E00E94F201892B51F4BE01EF
S11301806B5F7F4F84E592E00E94AC018D810E94F9
S11301906C000F900F900F900F900F90DF91CF9104
S11301A0FF91EF91BF91AF919F918F917F916F914B
S11301B05F914F913F912F910F900FBE0F901F9021
S11301C01895CF93DF931F92CDB7DEB789838091C3
S11301D0520290915302892B21F489810E946C0070
S11301E007C0BE016F5F7F4F84E592E00E94630108
S11301F00F90DF91CF910895F894809165029091CA
S11302006602019690936602809365020895809138
S1130210650290916602892B81F08091650290912C
S1130220660201979093660280936502809165024D
S113023090916602892B09F4789408958F929F9285
S1130240AF92BF92CF92DF92EF92FF920F931F93E0
S1130250CF93DF93EC017B014A015901198618867B
S11302601B861A861F821E827B836A835D834C836E
S1130270CB01880F991F0E94DD089983888300E0D1
S113028010E00E151F0581F0C801880F991FC88062
S1130290D980C80ED91EC4010E94DD08F6019183DD
S11302A080830F5F1F4FEDCFBD86AC86DF91CF916A
S11302B01F910F91FF90EF90DF90CF90BF90AF9080
S11302C09F908F9008950F931F93CF93DF93EC012A
S11302D08B010E94FC002E813F818A819B8128171B
S11302E0390768F5D8019D01201B310B8C819D8154
S11302F02817390780F4E885F9854D91EE0FFF1F23
S113030088819981E80FF91F80819181FC01E20FB6
S1130310F31F4083E8CF888599850196998788875C
S11303208E819F8101969F838E83288539858A815A
S11303309B812817390731F41986188603C0C0E059
S1130340D0E002C0C1E0D0E00E940701CE01DF91FD
S1130350CF911F910F9108950F931F93CF93DF9324
S1130360EC018B010E94FC008E819F81892B69F135
S1130370D801CD01801B910B2C813D8182179307FD
S113038080F4EA85FB85EE0FFF1F28813981E20F97
S1130390F31F20813181F901E80FF91F80818D93CA
S11303A0E8CF8A859B8501969B878A878E819F816A
S11303B001979F838E832A853B858A819B81281799
S11303C0390731F41B861A8603C0C0E0D0E002C0AE
S11303D0C1E0D0E00E940701CE01DF91CF911F91CF
S11303E00F910895CF93DF93EC010E94FC000E80DF
S11303F0DF81C02D0E94070181E090E0CD2B11F038
S113040080E090E0DF91CF9108958FEF8093B80062
S11304101092B900089594EA9093BC009091BC00A6
S113042097FFFCCF9091B900987F983019F081E242
S113043091E017C0880F682B6093BB0084E8809319
S1130440BC008091BC0087FFFCCF8091B900887FFD
S1130450883129F4FA01240F351F94E805C081E39B
S113046091E00E94770B14C0E217F30789F08191A1
S11304708093BB009093BC008091BC0087FFFCCFAD
S11304808091B900887F883279F383E491E0E9CFE1
S113049084E98093BC0008950F931F93CF93DF9357
S11304A000D000D0CDB7DEB78C0190936C0280935E
S11304B06B028091140190911501A0911601B091E5
S11304C0170189839A83AB83BC83809173029091D3
S11304D07402892BE9F0E1E0F0E00115110511F453
S11304E0E0E0F0E0EE0FFF1F81E090E08C0F9D1F35
S11304F0E80FF91F81818F9380818F9386E591E0C6
S11305009F938F930E94610B0F900F900F900F9009
S113051061E070E0012B11F460E070E087E090E0AE
S11305200F900F900F900F90DF91CF911F910F912B
S11305300C94B9060F931F93CF93DF9300D0CDB7DC
S1130540DEB78C0180936702109368028091730276
S113055090917402892B61F01F930F938FE691E0C1
S11305609F938F930E94610B0F900F900F900F90A9
S113057019821A8242E050E0BE016F5F7F4FC801CA
S11305800E949D069C01AE014F5F5F4F60E080E6D4
S11305900E940B020F900F90DF91CF911F910F914A
S11305A00895CF93DF93CDB7DEB76B970FB6F8946A
S11305B0DEBF0FBECDBFF894A8950FB6F894A895EA
S11305C080916000886180936000109260000FBE8B
S11305D02CE131E044E050E068E070E08DEB92E023
S11305E00E941E0140E052EC61E070E08DEB92E06D
S11305F00E94D50742E06FEF76EF8DEB92E00E9408
S11306004D078DEB92E00E9453000E9405020E9468
S1130610B10686E091E09093D2028093D10286E203
S113062092E09F938F938BE292E09F938F9387E85E
S113063091E09F938F930E94610B1D8A1E8A1F8AEB
S113064043E050E0BE016B5E7F4F80E090E00E948B
S1130650A4069C01AE014B5E5F4F60E080E60E9401
S11306600B026091D1027091D2028DE090E00E9461
S1130670250B6091D1027091D2028AE090E00E9431
S1130680250B6091D1027091D2028AE390E00E941E
S1130690250B60E070E080E00E94650760E070E098
S11306A082E00E94650781E090E00E944C02789409
S11306B00F900F900F900F900F900F90F12C212C12
S11306C0312C68EE462E63E0562E612C712C74EBAF
S11306D0872E71E0972EEEEACE2EE1E0DE2E8DEB32
S11306E092E00E94F201892B09F022C3BE016F5EE1
S11306F07F4F8DEB92E00E94AC018989823009F42E
S11307002DC2833009F458C2813009F011C38A899B
S11307102091750230917602AE014F5F5F4FFA016E
S1130720E20FF31F10828D3009F003C2598F488FF6
S11307301092760210927502EF2C8F2D90E0880FA4
S1130740991F9C01205E3D4F3B8F2A8F56E9A52EB1
S113075051E0B52E088D198DF80180818823D9F0D8
S113076090E00E941D0B9C01C8010196998F888F0F
S11307702035310509F055C0F80121812F3329F4C2
S11307800E5F1F4F198F088F31C030E0205331099D
S11307902A303105F0F060E177E281E00E946507DC
S11307A06091D1027091D2028DE090E00E94250BFD
S11307B06091D1027091D2028AE090E00E94250BF0
S11307C06091D1027091D2028AE390E00E94250BDD
S11307D06FC24AE050E0BE01685E7F4F0E94FE098E
S11307E0E1E0FE12C3C0CB010E949A026091D102E3
S11307F07091D2028DE090E00E94250B6091D102AD
S11308007091D2028AE090E00E94250B80916802E8
S11308108F93809167028F932EE831E03F932F935B
S113082068C123353105B1F5F80121812F3329F44D
S11308300E5F1F4F198F088F14C030E02053310909
S11308402A30310508F0A7CF4AE050E0BE01685EC7
S11308507F4F0E94FE09E1E0FE1288C0CB010E9496
S11308604C026091D1027091D2028DE090E00E941E
S1130870250B6091D1027091D2028AE090E00E942F
S1130880250B80916C028F9380916B028F9328EAE1
S113089031E0C4CF2235310509F07BC0F801218154
S11308A02F3309F47EC030E0205331092A3031055A
S11308B008F071CF4AE050E0BE01685E7F4F0E94AD
S11308C0FE096130710541F5F11050C08FEF9FE0D2
S11308D00E949A0280E090E00E944C026091D10252
S11308E07091D2028DE090E00E94250B6091D102BC
S11308F07091D2028AE090E00E94250B1F92F1E0F1
S1130900FF93DF92CF920E94610B0F900F900F9094
S11309100F90EE24E3941ECF672B09F01BCF21E048
S1130920F21224C08FEF9FE00E949A0280E090E0D0
S11309300E944C026091D1027091D2028DE090E04D
S11309400E94250B6091D1027091D2028AE090E05E
S11309500E94250B1F921F92DF92CF920E94610B7F
S11309600F900F900F900F90E12CF4CE6091D10274
S11309707091D2028DE090E00E94250B6091D1022B
S11309807091D2028AE090E00E94250BBF92AF9250
S1130990CBC02434310509F048C0F80121812F333C
S11309A0C9F40E5F1F4F198F088F6091D1027091A7
S11309B0D2028DE090E00E94250B6091D1027091EB
S11309C0D2028AE090E00E94250B81E0E81280E0E8
S11309D01F9227C030E0205331092A30310508F036
S11309E0DACE4AE050E0BE01685E7F4F0E94FE0905
S11309F070937402609373026091D1027091D20279
S1130A008DE090E00E94250B6091D1027091D2029A
S1130A108AE090E00E94250B809174028F9380916C
S1130A2073028F93DF92CF9264C029343105E1F4CD
S1130A30F80181818F3309F08DCE0E5F1F4F198F1E
S1130A40088F6091D1027091D2028DE090E00E94F3
S1130A50250B6091D1027091D2028AE090E00E944D
S1130A60250B2BE232E01EC026353105F1F4F801E6
S1130A7081818F3309F06ECE0E5F1F4F198F088F5F
S1130A806091D1027091D2028DE090E00E94250B1A
S1130A906091D1027091D2028AE090E00E94250B0D
S1130AA026E232E03F932F9322C02435310541F5ED
S1130AB0F80181818F3309F04DCE0E5F1F4F198FDE
S1130AC0088FEA8DFB8D108101816091D1027091B4
S1130AD0D2028DE090E00E94250B6091D1027091CA
S1130AE0D2028AE090E00E94250B0F931F939F92FD
S1130AF08F920E94610B0F900F900F900F902ACE4F
S1130B006091D1027091D2028DE090E00E94250B99
S1130B106091D1027091D2028AE090E00E94250B8C
S1130B202AEB31E03F932F930E94610B0F900F90BB
S1130B3011CE8A3009F4FCC02F30310538F42F5F10
S1130B403F4F309376022093750280836091D102E7
S1130B507091D20290E00E94250BEAC08A890B8929
S1130B601C89811116C08091690290916A0208174C
S1130B70190709F4DDC0F11007C0C801880F991FD7
S1130B80880F991F0E949A0210936A0200936902C7
S1130B90CFC0823009F0CCC010937202009371026E
S1130BA081E090E00130124014F480E090E09093F2
S1130BB0700280936F02BCC08A89813049F118F0B9
S1130BC08230A9F1B5C021E0F21203C024EF31E074
S1130BD002C028EE33E0810181E00827232819F4BC
S1130BE062E370E00BC022533109A8EEB3E00E9427
S1130BF0C308A30192010E94A108B90180E00E94E8
S1130C006507B80180E090E00E94B906180190C021
S1130C1091E0F9128DC08091730290917402892B36
S1130C2009F488C08EEC91E00E94770B83C062E3E4
S1130C3070E082E00E94650780916F0290917002DB
S1130C4020916D0230916E028217930711F1209169
S1130C50730230917402232B61F09F938F938EED76
S1130C6091E09F938F930E94610B0F900F900F90D0
S1130C700F9080916F0290917002892B51F48FEF45
S1130C808F0D823030F481E090E00E944C02E12C20
S1130C9001C0EF2C80916F029091700290936E02CC
S1130CA080936D0280E00E94E10082E00E94E100F6
S1130CB0FE14E1F18091730290917402892B01F189
S1130CC0EE2DF0E0EE0FFF1FE05EFD4F81818F936C
S1130CD080818F93EF2DF0E0EE0FFF1FE05EFD4F5C
S1130CE081818F9380818F9381EF91E09F938F9384
S1130CF00E94610B0F900F900F900F900F900F9028
S1130D00E2E0EE120BC08FEF9FE00E949A0280E0B7
S1130D1090E00E944C0261E070E004C0E11006C063
S1130D2060E070E082E090E00E94B906FE2CD7CC2F
S1130D30EF2CFCCF82E0E82EBDCF9F70FB019083A7
S1130D40818382E090E00895FB0120E4208324E085
S1130D50880F991F2A95E1F79183828383E090E0BD
S1130D6008958CEF8AB996E094B98BB984E085B97B
S1130D700895FC01EE0FFF1F8E0F9F1FFC01E75C1F
S1130D80FD4F808121E030E0018002C0220F331F3B
S1130D900A94E2F7428150E0E82FF0E080A1461780
S1130DA0570711F0282B02C02095282320A308956B
S1130DB01F920F920FB60F921124DF92EF92FF92BF
S1130DC00F931F932F933F934F935F936F937F934F
S1130DD08F939F93AF93BF93EF93FF93CF93DF933F
S1130DE000D000D0CDB7DEB78091B9029091BA029D
S1130DF09093850080938400E12CF12C93E0D92E0C
S1130E008701000F111F000F111F07581D4FF80114
S1130E1080819181892BF1F082819381892B31F03A
S1130E208281938101979383828314C019821A82E9
S1130E301B821C82D982EA82BE016F5F7F4F809140
S1130E407702909178020E946301892B19F0F801CE
S1130E5011821082FFEFEF1AFF0A80E1E816F10415
S1130E6079F60F900F900F900F90DF91CF91FF9133
S1130E70EF91BF91AF919F918F917F916F915F910E
S1130E804F913F912F911F910F91FF90EF90DF9021
S1130E900F900FBE0F901F90189590937802809337
S1130EA077027093BA026093B902709385006093DD
S1130EB0840010928000E1E8F0E080818770482B84
S1130EC0408381E080936F0008950F931F93CF9325
S1130ED0C82F8B010E94FC0084E0C89FF0011124FC
S1130EE0E758FD4F1383028381E090E09183808370
S1130EF0CF911F910F910C9407011F920F920FB67F
S1130F000F9211240F900FBE0F901F9018951F92EF
S1130F100F920FB60F9211240F900FBE0F901F90D7
S1130F2018951F920F920FB60F9211242F933F938F
S1130F304F935F936F937F938F939F93AF93BF93DD
S1130F40EF93FF93CF93DF9300D000D0CDB7DEB7FC
S1130F508091C00087FF12C08091C60019821A8256
S1130F601B821C8291E099838A83BE016F5F7F4F4D
S1130F708091BB029091BC020E9463010F900F907C
S1130F800F900F90DF91CF91FF91EF91BF91AF91AF
S1130F909F918F917F916F915F914F913F912F918D
S1130FA00F900FBE0F901F9018954F925F926F9203
S1130FB07F928F929F92AF92BF92CF92DF92EF92E5
S1130FC0FF92CF93DF9300D000D0CDB7DEB76A0194
S1130FD07B019093BC028093BB024A015B0183E0D6
S1130FE0880C991CAA1CBB1C8A95D1F760E070E898
S1130FF08CEF9AE0A50194010E94A108CA01B901ED
S11310006B5F7F4F8F4F9F4F2AE0422E512C612CF4
S1131010712CA30192010E94A10829833A834B8376
S11310205C8334E0CC0CDD1CEE1CFF1C3A95D1F73C
S113103060E070E88CEF9AE0A70196010E94A10895
S1131040CA01B9016B5F7F4F8F4F9F4FA30192017C
S11310500E94A10829013A01A501940169817A81BC
S11310608B819C810E949108705477FF03C0719515
S1131070619571094B01770FAA08BB08A701960176
S1131080C301B2010E949108705477FF03C07195A7
S113109061957109CB01770FAA0BBB0B88169906D2
S11310A0AA06BB0610F0920107C029813A818091FB
S11310B0C00082608093C000215031092093C40095
S11310C03093C50088E18093C1008091C10080689D
S11310D08093C1000F900F900F900F90DF91CF91EC
S11310E0FF90EF90DF90CF90BF90AF909F908F9044
S11310F07F906F905F904F9008959091C00095FFFE
S1131100FCCF8093C6000895CF93C82F0E947D081A
S1131110CA3019F48DE00E947D0880E090E0CF9100
S11311200895DB018F939F930E94D208BF91AF91E2
S1131130A29F800D911DA39F900DB29F900D11242D
S11311400895A1E21A2EAA1BBB1BFD010DC0AA1F04
S1131150BB1FEE1FFF1FA217B307E407F50720F01C
S1131160A21BB30BE40BF50B661F771F881F991F97
S11311701A9469F760957095809590959B01AC01E0
S1131180BD01CF010895A29FB001B39FC001A39FE9
S1131190700D811D1124911DB29F700D811D1124AC
S11311A0911D08950E94C308A59F900DB49F900DB2
S11311B0A49F800D911D112408950F931F93CF9325
S11311C0DF938230910510F482E090E0E091CD024B
S11311D0F091CE0220E030E0A0E0B0E0309719F1C9
S11311E0408151810281138148175907C8F084173F
S11311F0950769F4109731F012960C931297139691
S11312001C9327C00093CD021093CE0222C0211557
S1131210310519F04217530718F49A01BD01EF0183
S1131220DF01F801DBCF21153105F9F0281B390B5B
S11312302430310580F48A819B816115710521F088
S1131240FB019383828304C09093CE028093CD02EA
S1131250FE01329644C0FE01E20FF31F8193919385
S113126022503109398328833AC02091CB0230912E
S1131270CC02232B41F420910201309103013093DD
S1131280CC022093CB022091000130910101211561
S1131290310541F42DB73EB7409104015091050149
S11312A0241B350BE091CB02F091CC02E217F3073B
S11312B0A0F42E1B3F0B2817390778F0AC014E5FC2
S11312C05F4F2417350748F04E0F5F1F5093CC0231
S11312D04093CB028193919302C0E0E0F0E0CF0110
S11312E0DF91CF911F910F910895CF93DF930097D2
S11312F009F481C0FC01329713821282A091CD02BD
S1131300B091CE02109781F420813181820F931F16
S11313102091CB023091CC022817390751F5F09374
S1131320CC02E093CB0267C0ED0120E030E0CE17A1
S1131330DF0740F44A815B819E0141155105F1F0BC
S1131340EA01F5CFD383C28340815181840F951F75
S1131350C817D90759F488819981840F951F02967B
S1131360918380838A819B819383828321153105B4
S113137029F4F093CE02E093CD023DC0E901FB8352
S1131380EA8349915991C40FD51FEC17FD0761F405
S113139080819181840F951F0296E9019983888346
S11313A0828193819B838A83E0E0F0E012968D91A1
S11313B09C911397009719F0FD01DC01F7CF8D91F3
S11313C09C9111979D012E5F3F4F820F931F209197
S11313D0CB023091CC022817390769F4309729F4ED
S11313E01092CE021092CD0202C013821282B093E8
S11313F0CC02A093CB02DF91CF910895A0E0B0E09E
S1131400E4E0FAE00C94000E5C016B017A016115D2
S1131410710519F0FB0191838083E114F10429F033
S1131420C7010297839708F0E5C0E5012196F5010D
S11314301081812F90E00E94140B892B11F05E0122
S1131440F4CF1D3229F42196F501118101E007C082
S11314501B3221F4E5012296F501118100E0E1142B
S1131460F10409F1F0E1EF16F10429F43FC010E3AF
S1131470E114F10421F128E0E216F10401F154F43D
S1131480E2E0EE16F10421F5812C912CA12CB0E4BC
S1131490BB2E3EC0FAE0EF16F10439F020E1E2166B
S11314A0F104B1F430C0103319F1FAE0EF2EF12C4D
S11314B0ACEC8A2E982CA82CACE0BA2E29C078E08B
S11314C0E72EF12C812C912CA12CE0E1BE2E20C022
S11314D060E070E080E090E897010F2C000C440B72
S11314E0550B0E94A10849015A0112C0103359F446
S11314F088818F7D883509F0BACF198122960260E0
S113150080E1E82EF12C812C912CA12C68E0B62EE0
S113151040E060E070E0CB0127010F2C000C66086E
S11315207708FE0150ED352E310E29E0231570F4B5
S11315302FEB210F2A3118F439EC332E06C02FE992
S1131540210F2A3118F529EA322E310E232D30E0ED
S11315502E153F05DCF447FD16C086169706A8062F
S1131560B90670F0A30192010E949108630D711DE8
S1131570811D911D61307105810520E8920710F0ED
S11315804FEF01C041E021961081CBCF202F217075
S1131590C114D10471F0442329F02197F601D183B9
S11315A0C08307C001FF19C02297F601D183C0830D
S11315B014C047FF12C0222329F060E070E080E0ED
S11315C090E804C06FEF7FEF8FEF9FE722E230E0F7
S11315D03093D6022093D50209C0222381F090953E
S11315E08095709561957F4F8F4F9F4F462F372F72
S11315F0282F12C040E030E020E090E00DC097FFBB
S1131600F5CF82E290E09093D6028093D5026FEFFB
S11316107FEF8FEF9FE7EACF642F732F822FCDB731
S1131620DEB7E1E10C941C0E91110C94880D80320C
S113163019F089508550C8F708959111089581567D
S11316408A5108F48052855808950F931F93CF93BD
S1131650DF93FB01238121FD03C08FEF9FEF2CC09B
S113166022FF16C0468157812481358142175307D2
S113167044F4A081B1819D012F5F3F4F31832083CA
S11316808C93268137812F5F3F4F3783268314C085
S11316908B01EC01FB010084F185E02D0995892B78
S11316A0E1F6D80116968D919C911797019617969D
S11316B09C938E931697CE01DF91CF911F910F913A
S11316C00895A0E0B0E0E7E6FBE00C940F0EAE0155
S11316D04B5F5F4FFA0161917191AF018091D1022B
S11316E09091D2020E94A70BE2E00C942B0E0F9370
S11316F01F93CF93DF93E091D102F091D202238123
S113170021FF1BC08C01D0E0C0E0F80181918F0162
S11317106091D1027091D202DB011896ED91FC9197
S11317201997882331F00995892B79F3DFEFCFEFEF
S1131730ECCF8AE00995892B19F08FEF9FEF02C057
S11317408D2F9C2FDF91CF911F910F910895ABE0C6
S1131750B0E0EDEAFBE00C94FF0D6C017B018A0123
S1131760FC0117821682838181FFCCC1CE010196D0
S11317703C01F6019381F70193FD859193FF8191DB
S11317807F01882309F4BAC1853239F493FD859128
S113179093FF81917F01853229F4B60190E00E9484
S11317A0250BE7CF912C212C312CFFE1F315D8F038
S11317B08B3279F038F4803279F08332A1F4232D1E
S11317C020611DC08D3261F0803369F4232D2160C6
S11317D016C0832D8260382EE32DE4603E2E2AC08D
S11317E0F32DF8601DC037FC2DC020ED280F2A30E2
S11317F040F08E32B9F436FC81C1232D2064322EA0
S113180019C036FE06C08AE0989E200D1124922E3F
S113181011C0EAE02E9E200D1124222EF32DF06239
S11318203F2E08C08C3621F4832D8068382E02C0E8
S1131830883641F4F70193FD859193FF81917F01EF
S11318408111B3CF982F9F7D9554933028F40C5F6A
S11318501F4F9FE399830DC0833631F0833771F0B6
S1131860833509F059C021C0F801808189830E5F56
S11318701F4F88248394912C530113C02801F2E054
S11318804F0E511CF801A080B18036FE03C0692DB3
S113189070E002C06FEF7FEFC5010E94960D4C010E
S11318A08201F32DFF773F2E16C0280122E0420E5D
S11318B0511CF801A080B18036FE03C0692D70E090
S11318C002C06FEF7FEFC5010E948B0D4C01F32D19
S11318D0F0683F2E820133FC1BC0822D90E08816F5
S11318E09906B0F4B60180E290E00E94250B2A9498
S11318F0F4CFF50137FC859137FE81915F01B60184
S113190090E00E94250B21102A9421E0821A91086C
S11319108114910471F7E8C0843611F0893641F5D9
S1131920F80137FE07C060817181828193810C5F69
S11319301F4F08C060817181072E000C880B990B22
S11319400E5F1F4FF32DFF763F2E97FF09C0909532
S11319508095709561957F4F8F4F9F4FF0683F2E14
S11319602AE030E0A3010E94A10D882E861845C00C
S1131970853731F4232D2F7EB22E2AE030E025C0A6
S1131980932D997FB92E8F36C1F018F4883579F0EC
S1131990B5C0803719F0883721F0B0C0E92FE06175
S11319A0BE2EB4FE0DC0FB2DF460BF2E09C034FE64
S11319B00AC0292F2660B22E06C028E030E005C0F8
S11319C020E130E002C020E132E0F801B7FE07C0B8
S11319D060817181828193810C5F1F4F06C0608199
S11319E0718180E090E00E5F1F4FA3010E94A10D62
S11319F0882E8618FB2DFF773F2E36FE0DC0232D33
S1131A002E7FA22E891458F434FE0BC032FC09C078
S1131A10832D8E7EA82E05C0B82CA32C03C0B82C11
S1131A2001C0B92CA4FE0FC0FE01E80DF11D808198
S1131A30803321F49A2D997EA92E09C0A2FE06C0F6
S1131A40B394B39404C08A2D867809F0B394A3FCAC
S1131A5011C0A0FE06C0B21488F4280C922C9B1866
S1131A600EC0B21460F4B60180E290E00E94250B2F
S1131A70B394F7CFB21418F42B1802C0982C212C6D
S1131A80A4FE10C0B60180E390E00E94250BA2FEE4
S1131A9017C0A1FC03C088E790E002C088E590E08D
S1131AA0B6010CC08A2D867859F0A1FE02C08BE2E3
S1131AB001C080E2A7FC8DE2B60190E00E94250BF4
S1131AC0891438F4B60180E390E00E94250B9A94BF
S1131AD0F7CF8A94F301E80DF11D8081B60190E0FF
S1131AE00E94250B8110F5CF222009F442CEB601C5
S1131AF080E290E00E94250B2A94F6CFF6018681BD
S1131B00978102C08FEF9FEF2B96E2E10C941B0E9E
S1131B10992788270895FC010590615070400110B1
S1131B20D8F7809590958E0F9F1F0895FC01615002
S1131B30704001900110D8F7809590958E0F9F1FEB
S1131B400895FA01AA27283051F1203181F1E8944F
S1131B506F936E7F6E5F7F4F8F4F9F4FAF4FB1E09C
S1131B603ED0B4E03CD0670F781F891F9A1FA11D97
S1131B70680F791F8A1F911DA11D6A0F711D811D98
S1131B80911DA11D20D009F468943F912AE0269F5D
S1131B9011243019305D3193DEF6CF010895462FBC
S1131BA04770405D4193B3E00FD0C9F7F6CF462F9D
S1131BB04F70405D4A3318F0495D31FD4052419306
S1131BC002D0A9F7EACFB4E0A695979587957795C3
S1131BD06795BA95C9F700976105710508959B014A
S1131BE0AC010A2E06945795479537952795BA95D3
S1131BF0C9F7620F731F841F951FA01D08952F92AC
S1131C003F924F925F926F927F928F929F92AF9288
S1131C10BF92CF92DF92EF92FF920F931F93CF93D5
S1131C20DF93CDB7DEB7CA1BDB0B0FB6F894DEBF6C
S1131C300FBECDBF09942A88398848885F846E8492
S1131C407D848C849B84AA84B984C884DF80EE80DC
S1131C50FD800C811B81AA81B981CE0FD11D0FB6E5
S1131C60F894DEBF0FBECDBFED010895F894FFCF09
S1131C700000D702200000000002000000008408D9
S1131C800000000068016C01436F6E764669666F60
S1131C90004572726F72204932435F53544152546B
S1131CA0004572726F72204932435F534C415F4169
S1131CB0434B004572726F72204932435F44415472
S1131CC0415F41434B0053657420737769746368C3
S1131CD020746F2025730A004F4646004F4E005370
S1131CE0657420506F77657220746F2025752064A9
S1131CF069676974730A0025732025730A004F4BC2
S1131D003A25303475004552523A496E76616C6911
S1131D1064207374617465004F4B3A2575004F4B12
S1131D203A2564004F4B3A2573004552523A556E9A
S1131D306B6E6F776E20636F6D6D616E64005265BC
S1131D406D6F74652074696D656F757421005077CB
S1131D50725377697463685F696E203D2025640A55
S1131D60005374617465206368616E676520222581
S1131D707322203D3E20222573220A004E6F726D8D
S1131D80616C0052656D6F7465004572726F72000C
S1131D900C0213021A0276312E310048656E646912
S1131DA02D436F6E74726F6C000502010B06010BFC
S1131DB007010B02010B03010B04010B05010501D3
S1051DC001001C
S9030000FC
